:0E000000802EFF0226F6FFFFFFFFFF02241FE7
:030023000202488E
:20002E001A247581357508FF7509BF90AEBCE4F012496180EDC82581C822C92581C97A008F
:20004E0022D083D082CF2581F581CFC082C08322CF2581F581CF22FBE0CB22FCE0FBA3E06C
:20006E00CC22FAE0F9A3E0CA2229F9E5F03AFA227C00CB30E7011CCB2275F00030E70215FA
:20008E00F022FDE493A3FEE493A3FF4E7009E493FE740193FF800BE493A3B5050BE493B539
:2000AE00F0068F838E82E473A380D8FEEBA4FD8EF0ECA4FCEB8EF0A4C5F02C2DC5F0221131
:2000CE00D38EF0ED22C002C001AAF0F97E007D007F11C3E933F9EA33FADF08F5F0E9D0019C
:2000EE00D00222ED33FDEE33FEC3ED9BF5F0EE9C40E0ADF0FED380DBBB000122C333C5F096
:20010E0033C5F0DBF722BB000122C3C5F013C5F013DBF722240280022401C5F03400C5F065
:20012E0022C394028003C39401C5F09400C5F0223134F4C5F0F4C5F02245F0702204223144
:20014E00964024801A3196401E7014801A3196400E7014800A3196500E800431AA6008E4C7
:20016E00F5F02231AA60F8E4F5F0042231AA40F780ED31AA40F170E780ED31AA40E170E7A6
:20018E0080DD31AA50E180D7C39BC5F09C20E70720D207C345F02220D2F9D322C5F0C39CCD
:2001AE007003E5F09B2290AEBCE0A360EEE0FFA3E0A3CF2582F582EF3583F58380EB7E0067
:2001CE00CF2508F582EE3509F583EF227E00CF2508F9EE3509FAEF227E00C5082FC508C533
:2001EE00093EC50922E4F50AA88108E4F608B880FB22E4F520D201D200D203D205C2B4E4CB
:20020E00F50EF50DF50CF50BE4F512F511F510F50F74FFF513E588543FF588E589540FF512
:20022E00894420F5897450F598E5874480F58774FAF58BF58DD28ED2AC22C0E0C0D0C08365
:20024E00C082309839E50DB4FA028030502E050DE50DB50E0280044002F50E90A000C0E01B
:20026E00E50B2582F582E43583F583D0E0E599F0050BE50BB4FA004003750B00C29830999C
:20028E0048E511700DD200300235E4D5E0FDC2B4802DC20030011A300202D2B490A0FAC0F2
:2002AE00E0E5102582F582E43583F583D0E0E0F59915110510E510B4FA004003751000C2A3
:2002CE0099200105200002D299D082D083D0D0D0E0322278FB120043E6C0E0B40A0B300331
:2002EE0008D204740D1581C0E0E511B4FA0280F950F7C2AC90A0FAC0E0E50F2582F582E4C7
:20030E003583F583D0E0D0E0C0E0F00511050FE511B512004002F512E50FB4FA0040037525
:20032E000F00300002D299D2ACD0E0300408C204740AC0E080B322E4F5F078FB120043F6D9
:20034E0008A6F022E51364FF7038E50D6034300531C2AC90A000C0E0E50C2582F582E4357A
:20036E0083F583D0E0E0D2ACB40A0302038074018010150D050CE50CB4FA004003750C0085
:20038E0080C875F00022E4A20192E0F51F70030203B5E51160030203A0E4A20092E0F51F3C
:2003AE00E51F70030203A722C2AC7513FF7400F50CF50BC50DD2AC75F0002274FFC513B4AA
:2003CE00FF2EE50D0060FBC2AC90A000C0E0E50C2582F582E43583F583D0E0E0C0E0150DE2
:2003EE00050CE50CB4FA004003750C00D2ACD0E030050BB40A030203D0B40D02740A75F0D1
:20040E0000221203C9C0E0C0E0C0E01202E1D0E0D0E0D0E075F00022E51375F0007BFF7C0F
:20042E0000120169700302043E74FFF5F002044E78FB120043E60886F0F51318E60886F01F
:20044E002278FB1200438682088683E06016C083C082C0E0C0E01202E1D0E0D0E0D082D0F9
:20046E0083A380E722E4F5F078FB120043F608A6F02274B275F052C0E0C0F0E52075F000E1
:20048E00C0E0C0F07402124A8B158115811581158174CD75F052C0E0C0F0E50F75F000C0E8
:2004AE00E0C0F0E510C0E0C0F0E51175F000C0E0C0F0E512C0E0C0F0740575F000124A8BA2
:2004CE007FF612004F740075F053C0E0C0F0E50B75F000C0E0C0F0E50CC0E0C0F0E50D756F
:2004EE00F000C0E0C0F0E50EC0E0C0F0740575F000124A8B7FF612004FE4F50EF512227F41
:20050E00FD7EFF1201E8E4F5F07F001201CCF0A3C5F0F0C5F078FB120043E60886F0120105
:20052E003418F608A6F012012645F06022181818860108860289828A8312007089828A83CC
:20054E00E0120087C0E0C0F0124B841581158145F070030206197F001201CCE0A3F5F0E048
:20056E00C5F07B047C001201067F001201CCF0A3C5F0F0C5F078F9120043860108860289F3
:20058E00828A8312007089828A83E0120087C0E0C0F0124B93158115817F021201CCF07F70
:2005AE00021201CCE01200877B3912007E120153600B7F021201CCE0C39430800B7F0212D9
:2005CE0001CCE0C39441240A75F0007F001201CC1200692BC5F03CC5F07F001201CCF0A39A
:2005EE00C5F0F0C5F078F9120043860108860289828A83E0A3F5F0E0C5F012012689828AD3
:20060E0083F0A3C5F0F0C5F00205237F001201CCE0A3F5F0E0C5F07F030201E67FF17EFF7F
:20062E001201E87F021201DAE98AF0C0E0C0F0E4C0E0C0E0740A75F000C0E0C0F0124BC517
:20064E007FFA12004F7F021201DAE98AF07F0C1201CCF0A3C5F0F0C5F074097F0E1201CCA1
:20066E00F078FB120043860108860289828A8312007089828A83E0120087C0E0C0F0124BC5
:20068E004B1581158145F0602E78FB120043860108860289828A8312007089828A83E0128F
:2006AE000087C0E0C0F0124B7F1581158145F060067F0E1201CCE070030207397F0C120113
:2006CE00CCE0A3F5F0E0C5F01201267F0C1201CCF0A3C5F0F0C5F0120134F9AAF0C001C058
:2006EE000278F9120043860108860289828A8312007089828A83E0D083D082F0188601083F
:20070E00860289828A83E0A3F5F0E0C5F012012689828A83F0A3C5F0F0C5F07F0E1201CC84
:20072E00E0147F0E1201CCF002066F7F021201DAE98AF0C0E0C0F0124BE8158115817F00D3
:20074E001201CCF0A3C5F0F0C5F07F0F0201E67FFE7EFF1201E8E4F5F07F001201CCF0A399
:20076E00C5F0F0C5F07F001201CCE0A3F5F0E0C5F012014745F0601B78FB120043E6088670
:20078E00F012013418F608A6F01201267B007C0012015B45F0700302080378F7120043E66B
:2007AE000886F012012618F608A6F0120134F9AAF089828A83E0120087C0E0C0F008E60817
:2007CE0086F012012618F608A6F0120134F9AAF089828A83E0120087FBACF0D0F0D0E0C37B
:2007EE009BC5F09CC5F07F001201CCF0A3C5F0F0C5F00207737F001201CCE0A3F5F0E0C518
:20080E00F07F020201E67FFF7EFF1201E8E47F001201CCF07F001201CCE075F0007B107C9E
:20082E000012018070120208837F001201CCE0047F001201CCF080DC78FB120043E60886E0
:20084E00F07F001201CC1200652BC5F03400C5F0F9AAF07F001201CCE0C001C00279567A5F
:20086E00A412008712007789828A83E0F4D083D082F0020837740190A47AF07F010201E666
:20088E007FFF7EFF1201E8E4F521E4F5F090A2BEF0A3C5F0F0C5F0E490A2BDF074F475F024
:2008AE00A1C0E0C0F0E4C0E0C0E074C975F000C0E0C0F0124BC57FFA12004FE4F5F090A32B
:2008CE0089F0A3C5F0F0C5F074C075F0A2C0E0C0F0E4C0E0C0E074C975F000C0E0C0F012E1
:2008EE004BC57FFA12004FE490A455F0748C75F0A3C0E0C0F0E4C0E0C0E074C975F000C0C5
:20090E00E0C0F0124BC57FFA12004F740190A47AF0E47F001201CCF07F001201CCE075F055
:20092E00007B107C0012017A70120209947F001201CCE0047F001201CCF080DC7F00120176
:20094E00CCE079567AA41200871200777F001201CCE0C001C00279687AA4120087120077EC
:20096E0089828A83E0F4120087D083D08212006512007E1201717003020991E490A47AF023
:20098E0002099402093B90A47AE060030209D9745675F0A4C0E0C0F0E4C0E0C0E07412754D
:2009AE00F000C0E0C0F0124BC57FFA12004F745675F0A4C0E0C0F0745075F051C0E0C0F000
:2009CE00124C31158115811581158112175612175A746875F0A4C0E0C0F012081415811512
:2009EE00817F010201E612039478FB120043E60886F090A38BF0C209C2B490A38BE075F038
:200A0E0000900A32020090E490A38BF0D208C202E490AEBBF0020A46C208D202E490AEBBA0
:200A2E00F0020A46260A0300260A0200260A01001A0A00000000150A227FFB7EFF1201E879
:200A4E0078F9120043E60886F07F031201CCF0A3C5F0F0C5F008E60886F07F011201CCF055
:200A6E00A3C5F0F0C5F07F011201DAE98AF0C0E0C0F0740275F000C0E0C0F012050D158166
:200A8E001581158115817F001201CCF078FB120043E60886F0C0E0C0F0743075F000C0E013
:200AAE00C0F07402C0E0C0F0124BC57FFA12004F7F031201CC12007089828A83E070030266
:200ACE000B0A7F031201CC1200707F001201CCE089828A831200652B7F001201CCF07F0348
:200AEE001201CCE0A3F5F0E0C5F01201267F031201CCF0A3C5F0F0C5F0020ABE7F00120129
:200B0E00CCE0F4047F001201CCF078FB12004386010886027F001201CCE075F0007B047C58
:200B2E0000120114C001C00290515512007012007789828A83E0D083D082F078FB12004367
:200B4E00E60886F02401C5F03400C5F0F9AAF07F001201CCE0540FC001C002905155120061
:200B6E007012008712007789828A83E0D083D082F07F001201CCE012008754FFC5F0540015
:200B8E00C5F07F050201E690A455E06003020C3B748C75F0A3C0E0C0F0E4C0E0C0E074C957
:200BAE0075F000C0E0C0F0124BC57FFA12004F90A38BE075F0007B007C001201887003026C
:200BCE000C27798C7AA3742489828A83F0E4A20992E0F51F748C75F0A3C0E0C0F0E51F6041
:200BEE0007744475F0538005744875F053C0E0C0F0124C211581158115811581748C75F0EB
:200C0E00A3C0E0C0F0745675F0A4C0E0C0F0124C211581158115811581748C75F0A3C0E031
:200C2E00C0F0124C5F1581158190A455F078FB120043E60886F07B0A7C00120169700C1857
:200C4E00E60886F07BFF7C0012016945F07003020CCCE4A20992E0F51F7003020C8F748C09
:200C6E0075F0A3C0E0C0F0748C75F0A32401C5F03400C0F0C0E0120A47158115811581156E
:200C8E0081748C75F0A3C0E0C0F012044F1581158178FB120043E60886F07B0A7C0012019C
:200CAE00697003020CC4740A75F000C0E0C0F01202E115811581E490A455F0020CF8748CC1
:200CCE0075F0A390A4551200652BC5F03400C5F0F9AAF078FB120043E60886F089828A835E
:200CEE00F090A455E00490A455F02278FB120043860108860289828A83E07003020D3A1843
:200D0E00860108860289828A83E0120087C0E0C0F0120B951581158178FB120043E60886B3
:200D2E00F012012618F608A6F0020CF9227FFA7EFF1201E8E4F5F07F021201CCF0A3C5F045
:200D4E00F0C5F078FB120043E60886F07F001201CCF0A3C5F0F0C5F0E47F041201CCF07FB4
:200D6E00041201CCE075F0007B027C0012017A7003020FBB7F041201CCE075F000900F91A1
:200D8E00020090C2097F001201CCE0A3F5F0E0C5F01201267F001201CCF0A3C5F0F0C5F009
:200DAE00120134F9AAF089828A83E0120087900F080200907F001201CC12007089828A8389
:200DCE00E01200877B2012007E1201697003020DEA74017F041201CCF0020DF274037F04B7
:200DEE001201CCF0020F1478FB120043E60886F0C0E0C0F018E60886F02401C5F03400C02B
:200E0E00F0C0E0120A4715811581158115817F051201CCF07F051201CCE07003020EA87444
:200E2E00037F041201CCF0742F75F075C0E0C0F090A2BEE0A3F5F0E0C5F012012690A2BE6C
:200E4E00F0A3C5F0F0C0F0C0E0124CA6158115811581158190A2BEF0A3C5F0F0C5F090A390
:200E6E008BE075F0007B027C001201697003020EA5744A75F053C0E0C0F07F051201CCE0EE
:200E8E0075F000C0E0C0F0740275F000124A8B1581158115811581020EFA7F001201CCE02D
:200EAE00A3F5F0E0C5F02402C5F03400C5F07F001201CCF0A3C5F0F0C5F07F001201CC1288
:200ECE00007089828A83E01200877B2012007E1201697003020EF274017F041201CCF0D24E
:200EEE0009020EFA74037F041201CCF0020F1474037F041201CCF0020F14F50D2300C20D01
:200F0E0021000000FD0E020F9D745675F0A4C0E0C0F07F001201CCE0A3F5F0E0C0F0C0E0D0
:200F2E00745675F0A4C0E0C0F0124C5F15811581C0E0C0F012075D7FFA12004F45F070034F
:200F4E00020F5C74037F041201CCF0020F8E74027F041201CCF0745675F0A4C0E0C0F012B1
:200F6E004C5F158115817F001201CC1200692BC5F03CC5F07F021201CCF0A3C5F0F0C5F095
:200F8E00020F9D170F0100910D000000009D0F7F001201CCE0A3F5F0E0C5F01201267F0011
:200FAE001201CCF0A3C5F0F0C5F0020D6D7F021201CCE0A3F5F0E0C5F07F060201E67FFD94
:200FCE007EFF1201E8E4F5F07F011201CCF0A3C5F0F0C5F012035245F0700302126F1203CF
:200FEE00C97F001201CCF0E4A20892E0F51F70030210157F001201CCE0120087C0E0C0F0F7
:20100E001202E11581158190A2BDE0600302103D74F475F0A1C0E0C0F0E4C0E0C0E074C901
:20102E0075F000C0E0C0F0124BC57FFA12004F7F001201CCE01200879010B502009090A201
:20104E00BDE0700302106E90A2BDE01490A2BDF079F47AA1120087120077E489828A83F09A
:20106E000210C10210C174F475F0A190A2BD1200652BC5F03400C5F0F9AAF07F001201CC2E
:20108E00E089828A83F090A2BDE00490A2BDF075F0007BC87C0012019070030210B274C76F
:2010AE0090A2BDF00210C171100A004C100800000074107F001201CCE01200877B0A12008F
:2010CE007E120169700302126F90A38BE075F00090125602009079F47AA189828A83E012F3
:2010EE0000877B2A12007E120171700302110E74F475F0A17F011201CCF0A3C5F0F0C5F054
:20110E0002126A74F475F0A1C0E0C0F0120D3B158115817F011201CCF0A3C5F0F0C5F002B1
:20112E00126A90A2BDE070030211AD79F47AA189828A83E012008790119D0200900211AD7A
:20114E00746175F053C0E0C0F012044F1581158174F475F0A1C0E0C0F012044F15811581C4
:20116E00746375F053C0E0C0F012044F1581158174F475F0A1C0E0C0F0120D3B15811581AD
:20118E007F011201CCF0A3C5F0F0C5F00211AD4B112D004B112A004B11240000004E110245
:2011AE00126A90A2BDE0700302124079F47AA189828A83E01200879012300200900212403E
:2011CE0074F475F0A1C0E0C0F0120D3B158115817F011201CCF0A3C5F0F0C5F07F011201DE
:2011EE00CCE0A3F5F0E0C5F045F0700302122D746575F053C0E0C0F012044F158115817449
:20120E005675F0A4C0E0C0F012044F15811581746975F053C0E0C0F012044F158115810208
:20122E001240CB112D00CB112A00CB1124000000CE1102126A740175F000C0E0C0F012099D
:20124E00F41581158102126AB01103003011020011110100E410000000004312E490A2BD9C
:20126E00F07F011201CCE0A3F5F0E0C5F07F030201E690A38BE075F0007B007C0012016933
:20128E00700E90A38BE075F0007B027C0012016945F070030212B978FB120043E60886F0A9
:2012AE00C0E0C0F0120CF9158115812290A38BE075F0007B007C0012016970030212ED740D
:2012CE005675F0A4C0E0C0F012044F15811581746D75F053C0E0C0F012044F158115812224
:2012EE007FFD7EFF1201E878FB120043E60886F02401C5F03400C5F0F9AAF089828A83E072
:20130E001200877B3D12007E120169700302144918E60886F02402C5F03400C5F07F0012BF
:20132E0001CCF0A3C5F0F0C5F07F001201CCE0A3F5F0E0C0F0C0E0124C5F158115817B018A
:20134E007C001201637003021436745675F0A4C0E0C0F0E4C0E0C0E0741275F000C0E0C03C
:20136E00F0124BC57FFA12004FE47F021201CCF07F021201CCE075F0007B107C0012017A06
:20138E00600D7F001201CC12007089828A83E070120213F37F021201CCE0047F021201CCCC
:2013AE00F080CD7F021201CCE079567AA41200871200777F001201CCE0A3F5F0E0C5F01226
:2013CE0001267F001201CCF0A3C5F0F0C5F0120134C001C002F9AAF089828A83E0D083D015
:2013EE0082F00213A2745675F0A4C0E0C0F0745675F0A4C0E0C0F0124C5F15811581D004B3
:20140E00D0032BC5F03CC5F0F9AAF0742089828A83F0121756746875F0A4C0E0C0F012081D
:20142E001415811581021446746F75F053C0E0C0F012128015811581021494121756746842
:20144E0075F0A4C0E0C0F01208141581158174C075F0A2C0E0C0F0748975F053C0E0C0F03B
:20146E00745675F0A4C0E0C0F0740375F000124A9C7FFA12004F74C075F0A2C0E0C0F012F0
:20148E000CF9158115817F030201E678FB120043E60886F018F608A6F074C075F0A2C0E0EF
:2014AE00C0F0749C75F053C0E0C0F0745675F0A4C0E0C0F0740375F000124A9C7FFA1200D4
:2014CE004F74C075F0A2C0E0C0F0120CF915811581788018E660FC881F74C075F0A2C0E00D
:2014EE00C0F074AD75F053C0E0C0F0E51F75F000C0E0C0F0747FC0E0C0F0740475F000121A
:20150E004A9C7FF812004F74C075F0A2C0E0C0F0120CF9158115812278FB120043E60886D3
:20152E00F018F608A6F074C075F0A2C0E0C0F074C775F053C0E0C0F0E50A75F000C0E0C07F
:20154E00F090A2BEE0A3F5F0E0C0F0C0E0740475F000124A9C7FF812004F74C075F0A2C05D
:20156E00E0C0F0120CF915811581E4F50AE4F5F090A2BEF0A3C5F0F0C5F0227FFE7EFF12D3
:20158E0001E878FB120043E60886F02401C5F03400C5F07F001201CCF0A3C5F0F0C5F07F9B
:2015AE00001201CC12007089828A83E0120087C0E0C0F0124B7F1581158145F07003021514
:2015CE00EB7F001201CCE0A3F5F0E0C0F0C0E0124BE81581158190AEBBF002162574C075DC
:2015EE00F0A2C0E0C0F074F675F053C0E0C0F090AEBBE075F000C0E0C0F0740375F000120D
:20160E004A9C7FFA12004F74C075F0A2C0E0C0F0120CF9158115817F020201E67FFE7EFFCA
:20162E001201E878FB120043E60886F02401C5F03400C5F07F001201CCF0A3C5F0F0C5F067
:20164E007F001201CC12007089828A83E01200879016F902009074C075F0A2C0E0C0F074DB
:20166E000A75F054C0E0C0F090A38BE075F000C0E0C0F0740375F000124A9C7FFA12004F48
:20168E0074C075F0A2C0E0C0F0120CF9158115810217017F001201CC12007089828A83E07C
:2016AE00120087C0E0C0F0124B7F1581158145F070030216E67F001201CCE0A3F5F0E0C01F
:2016CE00F0C0E0124BE815811581C0E0C0F01209F4158115810216F6741A75F054C0E0C0BB
:2016EE00F012128015811581021701641600000000A1167F020201E690A38BE075F0007BE9
:20170E00007C00120169700302175574C075F0A2C0E0C0F0743275F054C0E0C0F078F71227
:20172E000043E60886F0C0E0C0F0740375F000124A9C7FFA12004F74C075F0A2C0E0C0F06B
:20174E001212801581158122E4F5F022D290A290B3E492E0F51FE51F700302177AE4C0E05F
:20176E00C0E01209F41581158102178A740175F000C0E0C0F01209F415811581227FFA7E5F
:20178E00FF1201E878FB120043E60886F07F021201CCF0A3C5F0F0C5F07F001201CCF0A3D7
:2017AE00C5F0F0C5F07F001201CC12007089828A83E070030218657F001201CC120070898E
:2017CE00828A83E01200877B2012007E12016970030218007F001201CCE0A3F5F0E0C5F064
:2017EE001201267F001201CCF0A3C5F0F0C5F00218627F021201CC120070C001C0027F00F7
:20180E001201CC12007089828A83E0120087C0E0C0F0124B9315811581D083D082F07F0048
:20182E001201CCE0A3F5F0E0C5F01201267F001201CCF0A3C5F0F0C5F07F021201CCE0A357
:20184E00F5F0E0C5F01201267F021201CCF0A3C5F0F0C5F00217B37F021201CC120070E4E8
:20186E0089828A83F078FB120043E60886F02401C5F03400C5F07F001201CCF0A3C5F0F0CD
:20188E00C5F018860108860289828A83E0120087901EF502009078FB120043E60886F0C0A4
:2018AE00E0C0F01212EE15811581021F2D12149912397F021F2D78FB120043E60886F0C03B
:2018CE00E0C0F012152615811581021F2D122A7C122A6C021F2D78FB120043E60886F0C009
:2018EE00E0C0F012158915811581021F2D7F001201CC12007089828A83E0120087C0E0C04F
:20190E00F0124B7F1581158145F070030219397F001201CCE0A3F5F0E0C0F0C0E0124BE88A
:20192E001581158190ACB4F002197374C075F0A2C0E0C0F0744D75F054C0E0C0F090ACB4BA
:20194E00E075F000C0E0C0F0740375F000124A9C7FFA12004F74C075F0A2C0E0C0F0120C8D
:20196E00F915811581021F2D78FB120043E60886F0C0E0C0F012162A15811581021F2DE4BA
:20198E00A21692E0F51F74C075F0A2C0E0C0F0746D75F054C0E0C0F0E51F75F000C0E0C0BD
:2019AE00F07403124A9C7FFA12004F74C075F0A2C0E0C0F0120CF915811581E4A21592E005
:2019CE00F51F74C075F0A2C0E0C0F0747675F054C0E0C0F0E51F75F000C0E0C0F074031225
:2019EE004A9C7FFA12004F74C075F0A2C0E0C0F0120CF915811581C215021F2D7F00120194
:201A0E00CC12007089828A83E0120087901B1702009074FF75F000C0E0C0F0E4C0E0C0F029
:201A2E001230801581158115811581021B2374FE75F000C0E0C0F0E4C0E0C0F0123080150C
:201A4E0081158115811581021B237F001201CC12007089828A83E07003021B147F001201E7
:201A6E00DAE98AF0C0E0C0F0121F32158115817F041201CCF0A3C5F0F0C5F07F041201CC8B
:201A8E00E0A3F5F0E0C5F012014745F0703A7F041201CCE0A3F5F0E0C5F07B027C00120197
:201AAE0069600E90A47CE075F0007BFF7C0012016945F070137F041201CCE0A3F5F0E0C5B3
:201ACE00F07B037C0012016945F07003021B0190A47BE075F000C0E0C0F090A47CE075F093
:201AEE0000C0E0C0F01230801581158115811581021B11747A75F054C0E0C0F01212801590
:201B0E00811581021A58021B233C1A5300201A00000000581A021F2D7F001201CC12007069
:201B2E0089828A83E0120087901C8802009074C075F0A2C0E0C0F0749275F054C0E0C0F0A6
:201B4E0090ACB5E0A3F5F0E0C0F0C0E0123E7AC0E0C0F0740475F000124A9C7FF812004F27
:201B6E0074C075F0A2C0E0C0F0120CF915811581021CA07F001201CCE0A3F5F0E0C5F0244C
:201B8E0001C5F03400C0F0C0E0124BE8158115817B3C7C001200B9C0E0C0F01246D415817C
:201BAE001581021CA07F001201CCE0A3F5F0E0C0F0C0E074B875F054C0E0C0F0124CED1538
:201BCE008115811581158145F07003021BEF74BD75F054C0E0C0F012128015811581021BD9
:201BEE00F5120394020000021CA0123F5F021CA07F001201CCE0A3F5F0E0C5F02401C5F0D6
:201C0E003400C0F0C0E0124BE815811581C0E0C0F01246AA15811581021CA07F001201CC27
:201C2E0012007089828A83E0120087C0E0C0F0124B7F1581158145F07003021C757F00125F
:201C4E0001CCE0A3F5F0E0C0F0C0E0124BE8158115817B3C7C001200B9C0E0C0F01246AA50
:201C6E0015811581021C8574D275F054C0E0C0F012128015811581021CA0FE1B5300F81B2B
:201C8E005100B31B4500811B43003C1B00000000291C021F2D7F001201CC12007089828A94
:201CAE0083E07003021D657F001201DAE98AF0C0E0C0F0121F32158115817F041201CCF0BC
:201CCE00A3C5F0F0C5F07F041201CCE0A3F5F0E0C5F045F07003021CFA74EA75F054C0E023
:201CEE00C0F012128015811581021D6290A47BE075F000C0E0C0F090A47CE075F000C0E0FC
:201D0E00C0F090A47DE075F000C0E0C0F090A47EE075F000C0E0C0F012361E7FF812004F3A
:201D2E0090A47BE075F000C0E0C0F090A47CE075F000C0E0C0F090A47DE075F000C0E0C0B6
:201D4E00F090A47EE075F000C0E0C0F01241217FF812004F021CA3021F2D021F2D740275AA
:201D6E00F055C0E0C0F0120CF915811581743875F055C0E0C0F0120CF915811581745B7540
:201D8E00F055C0E0C0F0120CF915811581749775F055C0E0C0F0120CF91581158174C1755B
:201DAE00F055C0E0C0F0120CF91581158174E875F055C0E0C0F0120CF91581158174177594
:201DCE00F056C0E0C0F0120CF915811581744575F056C0E0C0F0120CF915811581746575C7
:201DEE00F056C0E0C0F0120CF915811581749875F056C0E0C0F0120CF91581158174B87501
:201E0E00F056C0E0C0F0120CF91581158174E675F056C0E0C0F0120CF91581158174167534
:201E2E00F057C0E0C0F0120CF915811581743D75F057C0E0C0F0120CF9158115817462756F
:201E4E00F057C0E0C0F0120CF915811581748875F057C0E0C0F0120CF91581158174BC75AA
:201E6E00F057C0E0C0F0120CF91581158174E275F057C0E0C0F0120CF915811581740C75E0
:201E8E00F058C0E0C0F0120CF915811581744175F058C0E0C0F0120CF915811581747475F7
:201EAE00F058C0E0C0F0120CF91581158174AB75F058C0E0C0F0120CF91581158174CA7517
:201ECE00F058C0E0C0F0120CF915811581021F2D78FB120043E60886F0C0E0C0F012170620
:201EEE0015811581021F2D6B1D3F00681D0000A31C5300261B52000A1A51008D1950007688
:201F0E00194E00FB184D00E4184C00DB184600C4184500BB184400A41841000000DE1E7FBB
:201F2E00060201E67FFA7EFF1201E8E4F5F07F041201CCF0A3C5F0F0C5F0E4F5F07F001241
:201F4E0001CCF0A3C5F0F0C5F078FB120043860108860289828A83E0A3F5F0E0C5F07F0244
:201F6E001201CCF0A3C5F0F0C5F0740290A47EF074FF90A47CF07F021201CC12007089826F
:201F8E008A83E012008745F060267F041201CCE0A3F5F0E0C5F012014745F060137F001200
:201FAE0001CCE0A3F5F0E0C5F07B047C0012014D45F0700302223F7F001201CCE0A3F5F01D
:201FCE00E0C5F09022280200907F021201CC12007089828A83E01200877B4112007E120120
:201FEE006360187F021201CC12007089828A83E01200877B5012007E12015345F07003021A
:20200E00205D7F021201CC12007089828A83E0C3944190A47BF07F021201CCE0A3F5F0E07C
:20202E00C5F01201267F021201CCF0A3C5F0F0C5F07F001201CCE0A3F5F0E0C5F0120126C3
:20204E007F001201CCF0A3C5F0F0C5F002206E740175F0007F041201CCF0A3C5F0F0C5F06E
:20206E0002223C7F021201CCE0A3F5F0E0C0F0C0E01238791581158190A47CF07B007C0074
:20208E00120190600E90A47CE075F0007B107C0012017A45F070030220E67F021201CCE0A8
:2020AE00A3F5F0E0C5F02402C5F03400C5F07F021201CCF0A3C5F0F0C5F07F001201CCE0A6
:2020CE00A3F5F0E0C5F01201267F001201CCF0A3C5F0F0C5F00220F7740275F0007F0412C8
:2020EE0001CCF0A3C5F0F0C5F002223C7F021201CCE0A3F5F0E0C0F0C0E012387915811552
:20210E008190A47DF075F0007BFF7C00120171600E90A47DE075F0007B107C00120190455D
:20212E00F070030221727F021201CCE0A3F5F0E0C5F02402C5F03400C5F07F021201CCF028
:20214E00A3C5F0F0C5F07F001201CCE0A3F5F0E0C5F01201267F001201CCF0A3C5F0F0C585
:20216E00F0022183740375F0007F041201CCF0A3C5F0F0C5F002223C7F021201CC1200704E
:20218E0089828A83E0120087C0E0C0F0124B7F1581158145F070030222047F021201CCE038
:2021AE00A3F5F0E0C0F0C0E0124BE81581158190A47EF07F021201CC12007089828A83E06C
:2021CE00120087C0E0C0F0124B7F1581158145F070030222017F021201CCE0A3F5F0E0C5C6
:2021EE00F01201267F021201CCF0A3C5F0F0C5F00221C102220A740290A47EF07F0012019F
:20220E00CCE0A3F5F0E0C5F01201267F001201CCF0A3C5F0F0C5F002223C86210300FA203F
:20222E00020071200100D71F000000003C22021F847F021201CC12007089828A83E0120017
:20224E008745F060187F021201CC12007089828A83E01200877B2C12007E12017145F07069
:20226E00030222907F021201CCE0A3F5F0E0C5F01201267F021201CCF0A3C5F0F0C5F002B4
:20228E00223F7F021201CC12007089828A83E01200877B2C12007E12016970030222C87FCB
:2022AE00021201CCE0A3F5F0E0C5F01201267F021201CCF0A3C5F0F0C5F078FB120043865E
:2022CE00010886027F021201CCE0A3F5F0E0C5F089828A83F0A3C5F0F0C5F07F041201CC9B
:2022EE00E0A3F5F0E0C5F07F060201E6E4F523F522E4F514E490ACB3F074B375F0AAC0E0CC
:20230E00C0F0E4C0E0C0E0E475F001C0E0C0F0124BC57FFA12004F74B375F0ABC0E0C0F0BE
:20232E00E4C0E0C0E0E475F001C0E0C0F0124BC57FFA12004FE4F518743575F04FF51985F4
:20234E00F01AE51875F000C333C5F033C5F079357A4F12007789828A83E0A3F5F0E0C5F05B
:20236E00F51B85F01CE4F515E4F517F516D295742775F000C0E0C0F0E4C0E0C0E0740475FD
:20238E00F000C0E0C0F0124D237FFA12004F747F75F0A4C0E0C0F0E4C0E0C0E074F475F056
:2023AE0005C0E0C0F0124BC57FFA12004FE4F52EF52DF52CF52B747F75F0A4F52485F025A5
:2023CE00747375F0AAC0E0C0F0E4C0E0C0E0744075F000C0E0C0F0124BC57FFA12004FE43C
:2023EE00F531E4F535F534F533F532740190ACB4F0E58854CFF588E58954F0F5894401F557
:20240E0089E4F58AF58CD2B9D2A9D28CD288D2A822D294C0E0C0D0A212B392B3C28C851BB7
:20242E008A851C8CD28CC0F0C083C082C000E518B415004016430A02904F358582198583DD
:20244E001AE0F51BA3E0F51CE4F51825E02477F58274243400F583E0F5F0A3E0C0E0C0F0EC
:20246E00E527A2E7821392122224A524B024BA24BD24C024C524C824CB24D024F824FB2506
:20248E0002250C250F25122517251A251D2522254625C400000000B294B294A21E921F0239
:2024AE0026CFA2B5B3921EC2120226CF0226CF0226CFC2120226CF0226CF0226CFC2120217
:2024CE0026CF301322E52A33F52AE52933F529E52833F528E52733F527E52A92E0F52AC2BA
:2024EE0012E526600215260226CF0225DFA21E921F0226CFA2B5B3921EC2120226CF022602
:20250E00CF0226CFC2120226CF0226CF0226CFC2120226CF30131EE52A33F52AE52933F56B
:20252E0029E52833F528E52733F527E52A92E0F52AC21215260226CF201310E52D7003023C
:20254E0025C18524828525830225A1E52660030225C1852482852583E0430A106007530AB8
:20256E00EF14F0702EE52C04B4FE004001E4F52C75F006A4247FF582E5F034A4F58385825A
:20258E0024858325152DE52D7009C213C212D2960225C1A3E0F526A375F0047827E0F6A354
:2025AE0008D5F0F9E527A2E79212D213C296B29600B2960225DFB294751800904F3585824D
:2025CE001985831AB294B294D214D289B2940226DF301D05C21D02266AE531B40A0280047B
:2025EE004002740B25E090260C0531D21DA21EB01F92D5A21FB01E72D592D5A21F73801623
:20260E00801C80288030803880408053805B8063806B8073803E301F3E301E3B803E301FF0
:20262E0036201E33752F00753000803030D528E53033F530802630D51EE53033F530801C80
:20264E0030D514E53033F530801230D50AE53033F5308008430A04753100C21D0226CF3053
:20266E00D5F5E52F33F52F80F330D5EBE52F33F52F80E930D5E1E52F33F52F80DF30D5D754
:20268E00E52F33F52F80D530D5CDE52F33F52F90AA73E53225E02582F582E43583F583E54F
:2026AE002FF0A3E530F00534E534B5350280044002F5350532E532B420004003753200808B
:2026CE00960518851A83851982A3A385831A858219E0F51BA3E0F51CD000D082D083D0F0B6
:2026EE00D0D0D0E0C2943222D293C0E0C0F0C0D0C083C082A212B392B37400B51802801287
:20270E00F518904F3585831A858219E0F51BA3E0F51CD28DE515B402028004400274032551
:20272E00E090273373800680168040805B20140302279E75150175160075170102279E200F
:20274E0014120516751700E516B41E00404275150002279E7516000517E517B41E00403019
:20276E00D216D215C29575150280252014157517000516E516B41E004016751500C216D2AD
:20278E0095800D7516008008751500430A018000C214C2890514E514B43C004005751400AD
:2027AE00D217D082D083D0D0D0F0D0E0C293322274C075F0A2C0E0C0F074E675F058C0E082
:2027CE00C0F078F7120043E60886F02441C5F03400C0F0C0E018E60886F07B057C001200EB
:2027EE00B92404C5F03400C5F079657A4F12007789828A83E075F000C0E0C0F0740475F092
:20280E0000124A9C7FF812004F74C075F0A2C0E0C0F0120CF9158115812274C075F0A2C0EF
:20282E00E0C0F074EE75F058C0E0C0F078F7120043E60886F07B057C001200B92404C5F0BF
:20284E003400C5F079C67A4F12007789828A83E075F000C0E0C0F0740375F000124A9C7FF0
:20286E00FA12004F74C075F0A2C0E0C0F0120CF9158115812274C075F0A2C0E0C0F074F30D
:20288E0075F058C0E0C0F078F7120043E60886F0C333C5F033C5F079867A50120077898205
:2028AE008A83E0A3F5F0E0C0F0C0E0740375F000124A9C7FFA12004F74C075F0A2C0E0C01C
:2028CE00F0120CF9158115812278FB120043E60886F079B57A4F12007789828A83E0C3949A
:2028EE00411200872278FB120043E60886F079667A5012007789828A83E075F000227FFE74
:20290E007EFF1201E8E5347003022A4BE53375F000C333C5F033C5F079737AAA12007789FC
:20292E00828A83E0A3F5F0E0C5F07F001201CCF0A3C5F0F0C5F00533E533E53375F0007B6A
:20294E00207C00120190700302295CE4F5331534E53490AEBBE0540175F0007B007C001226
:20296E0001717003022A4874F675F058C0E0C0F0120CF9158115817F001201CCE0A3F5F070
:20298E00E0C5F05400C5F0540FC5F07B087C00120114C0E0C0F01228D715811581C0E0C060
:2029AE00F01227BE1581158174FF75F058C0E0C0F0120CF9158115817F001201CCE0A3F55D
:2029CE00F0E0C5F0541FC5F05400C5F07B007C00120114C0E0C0F01228F315811581C0E0CC
:2029EE00C0F012282815811581740575F059C0E0C0F0120CF9158115817F001201CCE0A3E0
:202A0E00F5F0E0C5F0541FC5F05400C5F07B007C00120114C0E0C0F01228F315811581C076
:202A2E00E0C0F012288315811581740875F059C0E0C0F0120CF915811581022A5B74FFF553
:202A4E00F07F001201CCF0A3C5F0F0C5F07F001201CCE0A3F5F0E0C5F07F020201E612292D
:202A6E000C7BFF7CFF1201716003022A6C22C2A9C2A8C212C213742775F000C0E0C0F0E4F4
:202A8E00C0E0C0E0740475F000C0E0C0F0124D237FFA12004F747F75F0A4C0E0C0F0E4C06F
:202AAE00E0C0E074F475F005C0E0C0F0124BC57FFA12004FE4F52EF52DF52CF52B747F7598
:202ACE00F0A4F52485F025D296D2A8D2A9227FFD7EFF1201E878FB120043E60886F05400AE
:202AEE00C5F0540FC5F07B087C0012011479B57A4F12007789828A83E0C394417F01120132
:202B0E00CCF078FB120043E60886F0541FC5F05400C5F07B007C0012011479667A501200B5
:202B2E007789828A83E07F001201CCF090ACB3E075F000902D110200907F001201CCE07583
:202B4E00F0007B107C0012017A7003022C09E47F021201CCF07F021201CCE075F0007B10D5
:202B6E007C0012017A7012022BD97F021201CCE0047F021201CCF080DC7F021201CCE07511
:202B8E00F0007F011201CC1200657C001201717003022BD67F021201CCE075F0007B107C3F
:202BAE00001200B979B37AAA120077E98AF0C0E0C0F0E4C0E0C0E0741075F000C0E0C0F053
:202BCE00124BC57FFA12004F022B787F011201CCE075F0007B107C001200B97F001201CC72
:202BEE001200652BC5F03400C5F079B37AAA120077740189828A83F0022C347F011201CC70
:202C0E00E075F000C0E0C0F07F001201CCE075F000C0E0C0F0122D22158115811581158165
:202C2E00740190ACB3F0022D1D7F001201CCE075F0007B107C0012017A7003022C9F74B348
:202C4E0075F0AAC0E0C0F0E4C0E0C0E0E475F001C0E0C0F0124BC57FFA12004F7F011201BA
:202C6E00CCE075F0007B107C001200B97F001201CC1200652BC5F03400C5F079B37AAA1263
:202C8E000077740189828A83F0E490ACB3F0022CC47F011201CCE075F000C0E0C0F07F000A
:202CAE001201CCE075F000C0E0C0F0122D221581158115811581022D1DE50A4408F50AE46F
:202CCE0090ACB3F074B375F0AAC0E0C0F0E4C0E0C0E0E475F001C0E0C0F0124BC57FFA1216
:202CEE00004F74B375F0ABC0E0C0F0E4C0E0C0E0E475F001C0E0C0F0124BC57FFA12004F36
:202D0E00022D1D372C0100472B00000000C72C7F030201E67FFF7EFF1201E878FB12004367
:202D2E00E60886F0903063020090E47F001201CCF07F001201CCE075F0007B107C0012017D
:202D4E007A7012022DF77F001201CCE0047F001201CCF080DC78F9120043E60886F07B10A2
:202D6E007C001200B97F001201CC1200652BC5F03400C5F079B37AAA12007789828A83E08F
:202D8E007003022DF478F9120043E60886F07B107C001200B97F001201CC1200652BC5F0DE
:202DAE003400C5F079B37AAB120077740289828A83F078F9120043E60886F0C0E0C0F07FCB
:202DCE00001201CCE075F000C0E0C0F008E60886F0C0E0C0F0740275F000C0E0C0F0124137
:202DEE00217FF812004F022D5402307BE47F001201CCF07F001201CCE075F0007B107C00C0
:202E0E0012017A7012022EB57F001201CCE0047F001201CCF080DC78F9120043E60886F09A
:202E2E007B107C001200B97F001201CC1200652BC5F03400C5F079B37AAA12007789828AA6
:202E4E0083E07003022EB278F9120043E60886F07B107C001200B97F001201CC1200652BB0
:202E6E00C5F03400C5F079B37AAB120077740289828A83F078F9120043E60886F0C0E0C0C4
:202E8E00F07F001201CCE075F000C0E0C0F008E60886F0C0E0C0F0E4C0E0C0E01241217F6E
:202EAE00F812004F022E1602307BE47F001201CCF07F001201CCE075F0007B107C001201C9
:202ECE007A7012022F777F001201CCE0047F001201CCF080DC78F9120043E60886F07B109F
:202EEE007C001200B97F001201CC1200652BC5F03400C5F079B37AAA12007789828A83E00E
:202F0E007003022F7478F9120043E60886F07B107C001200B97F001201CC1200652BC5F0DA
:202F2E003400C5F079B37AAB120077740189828A83F078F9120043E60886F0C0E0C0F07F4A
:202F4E00001201CCE075F000C0E0C0F008E60886F0C0E0C0F0740275F000C0E0C0F01241B5
:202F6E00217FF812004F022ED402307B78F9120043E60886F0C0E0C0F07F001201CCE0756C
:202F8E00F000C0E0C0F008E60886F0C0E0C0F0E4C0E0C0E01241217FF812004FE47F001242
:202FAE0001CCF07F001201CCE075F0007B107C0012017A701202303F7F001201CCE0047F5B
:202FCE00001201CCF080DC78F9120043E60886F07B107C001200B97F001201CC1200652BBC
:202FEE00C5F03400C5F079B37AAB12007789828A83E075F0007B007C0012017170030230CE
:20300E003C78F9120043E60886F07B107C001200B97F001201CC1200652BC5F03400C5F0CC
:20302E0079B37AAB120077740189828A83F0022FC674B375F0AAC0E0C0F0E4C0E0C0E0E4A6
:20304E0075F001C0E0C0F0124BC57FFA12004F02307B02307B7A2F1000B82E1300FA2D1568
:20306E0000FA2D1400382D1200000060307F010201E67FFC7EFF1201E878F9120043E608F0
:20308E0086F09033AB020090E4F5F078F9120043F608A6F078F9120043E60886F07B107C58
:2030AE000012017A70160230EE78F9120043E60886F012012618F608A6F080D878F91200E5
:2030CE0043E60886F0C0E0C0F074FF75F000C0E0C0F012308015811581158115810230B7C0
:2030EE000233B7E4F5F078F9120043F608A6F078F9120043E60886F07B107C0012017A7085
:20310E001602322478F9120043E60886F012012618F608A6F080D8E4F5F07F001201CCF0B5
:20312E00A3C5F0F0C5F0E4F5F078FB120043F608A6F078FB120043E60886F07B107C00121A
:20314E00017A70160231E478FB120043E60886F012012618F608A6F080D878F9120043E634
:20316E000886F07B107C001200B90826C5F00836C5F079B37AAB12007789828A83E075F0E4
:20318E00007B027C001201696007740175F0008003E4F5F07F021201CCF0A3C5F0F0C5F0D2
:2031AE007F021201CCE0A3F5F0E0C5F078FB12004386030886041201067F001201CC120038
:2031CE00694BC5F04CC5F07F001201CCF0A3C5F0F0C5F002315574C075F0A2C0E0C0F074A5
:2031EE000B75F059C0E0C0F07F001201CCE0A3F5F0E0C0F0C0E0740375F000124A9C7FFA65
:20320E0012004F74C075F0A2C0E0C0F0120CF915811581023112740A75F000C0E0C0F012E7
:20322E000B95158115810233B778FB120043E60886F07BFF7C00120169700302331774C037
:20324E0075F0A2C0E0C0F0741075F059C0E0C0F0181818E60886F02441C5F03400C0F0C00D
:20326E00E0740375F000124A9C7FFA12004F74C075F0A2C0E0C0F0120CF915811581E4F50B
:20328E00F078FB120043F608A6F078FB120043E60886F07B107C0012017A701602330478DD
:2032AE00FB120043E60886F012012618F608A6F080D878F9120043E60886F07B107C0012CC
:2032CE0000B90826C5F00836C5F079B37AAB12007789828A83E0794C7A51120087120077CD
:2032EE0089828A83E0120087C0E0C0F0120B95158115810232AD740A75F000C0E0C0F012DB
:20330E000B95158115810233A874C075F0A2C0E0C0F0741475F059C0E0C0F078F512004313
:20332E00E60886F02441C5F03400C0F0C0E008E60886F02401C5F03400C0F0C0E01818186B
:20334E00E60886F07B107C001200B90826C5F00836C5F079B37AAB12007789828A83E0750C
:20336E00F000C333C5F033C5F079467A5112007789828A83E0A3F5F0E0C0F0C0E07405750B
:20338E00F000124A9C7FF612004F74C075F0A2C0E0C0F0120CF9158115810233B7F130FE88
:2033AE00009630FF00000037327F040201E67FFF7EFF1201E878FB120043E60886F024021D
:2033CE00C5F03400C0F0C0E0746175F04FC0E0C0F0740475F000C0E0C0F0124D7C7FFA123A
:2033EE00004FE47F001201CCF07F001201CCE075F0007B047C0012017A70130234827F0059
:20340E001201CCE0047F001201CCF01480DB78FB120043E60886F02402C5F03400C5F07FAF
:20342E00001201CC1200652BC5F03400C5F0F9AAF078F7120043E60886F07B057C00120096
:20344E00B97F001201CC1200652BC5F03400C5F0C001C00279657A4F120077D083D082C0EF
:20346E0082C083E089828A831200654BD083D082F002340CE47F001201CCF07F001201CC58
:20348E00E075F0007B047C0012017A70130235127F001201CCE0047F001201CCF01480DB86
:2034AE0078FB120043E60886F02402C5F03400C5F07F001201CC1200652BC5F03400C5F070
:2034CE00F9AAF0181818E60886F07B057C001200B97F001201CC1200652BC5F03400C5F03A
:2034EE00C001C00279C67A4F120077D083D082C082C083E089828A831200654BD083D08221
:20350E00F002349E7F010201E67FFF7EFF1201E8E52D75F0007BFE7C0012019070030235C1
:20352E0046E50A4420F50AE52D75F0007BFE7C00120190600302353578F5120043E60886D1
:20354E00F0C0E0C0F008E60886F0C0E0C0F0E52B75F0007B067C001200B92400C5F0340017
:20356E00C5F0797F7AA4120077E98AF0C0E0C0F01233BC7FFA12004FE52B75F0007B067CE9
:20358E00001200B92400C5F03400C5F0797F7AA412007778FB120043E60886F089828A83AD
:2035AE00F0E52B75F0007B067C001200B92401C5F03400C5F0797F7AA412007778F91200EB
:2035CE0043E60886F089828A83F0052BE52BE52B75F0007BFE7C0012019070030235F0E463
:2035EE00F52B052DE52D7F001201CCF0E52E75F0007F001201CC1200657C0012017A700342
:20360E000236197F001201CCE0F52E7F010201E690AEBBE0540275F0007B007C0012017172
:20362E007003023723741F75F059C0E0C0F0120CF91581158178F5120043E60886F0C0E003
:20364E00C0F01227BE15811581742875F059C0E0C0F0120CF91581158178F7120043E608EA
:20366E0086F0C0E0C0F012282815811581742C75F059C0E0C0F0120CF91581158178F91274
:20368E000043E60886F0C0E0C0F01228281581158174C075F0A2C0E0C0F0743075F059C0EA
:2036AE00E0C0F078F7120043E60886F0C0E0C0F0740375F000124A9C7FFA12004F74C0759D
:2036CE00F0A2C0E0C0F0120CF91581158178F7120043E60886F0C0E0C0F0122883158115D7
:2036EE0081742075F000C0E0C0F0120B951581158178F9120043E60886F0C0E0C0F0122860
:20370E008315811581743C75F059C0E0C0F0120CF91581158178F5120043E60886F0C0E025
:20372E00C0F008E60886F0C0E0C0F0741675F000C0E0C0F07401C0E0C0F01235177FF81224
:20374E00004F78F5120043E60886F0C0E0C0F008E60886F0C0E0C0F0742075F000C0E0C081
:20376E00F07401C0E0C0F01235177FF812004F740175F000C0E0C0F078F9120043E60886EC
:20378E00F0C0E0C0F0124C8A158115811581158178FB120043F608A6F074FF75F000C0E0C7
:2037AE00C0F018E60886F0C0E0C0F0124CA6158115811581158178FB120043F608A6F018AF
:2037CE00E60886F07B017C00120169700302381078F5120043E60886F0C0E0C0F0080808B8
:2037EE00E60886F0C0E0C0F0742075F000C0E0C0F07401C0E0C0F01235177FF812004F02C1
:20380E00387878F5120043E60886F0C0E0C0F0080808E60886F0C0E0C0F0741675F000C0F9
:20382E00E0C0F008E60886F0C39401C5F09400C0F0C0E01235177FF812004F78F512004395
:20384E00E60886F0C0E0C0F0080808E60886F0C0E0C0F0742075F000C0E0C0F07401C0E07C
:20386E00C0F01235177FF812004F227FFD7EFF1201E874FFF5F07F011201CCF0A3C5F0F04F
:20388E00C5F0E47F001201CCF07F001201CCE075F0007B207C0012017A701302396E7F0041
:2038AE001201CCE0047F001201CCF01480DB7F001201CCE075F0007B037C001200B92400EE
:2038CE00C5F03400C5F079C67A50120077C001C00278F91200438601088602D083D082E0C5
:2038EE0012008789828A8312006512007E120169604C7F001201CCE075F0007B037C00122B
:20390E0000B92401C5F03400C5F079C67A5012007778FB120043E60886F02401C5F0340051
:20392E00C5F0C001C002F9AAF0D083D082E012008789828A8312006512007E12016945F0C0
:20394E00700302396B7F001201CCE075F0007F011201CCF0A3C5F0F0C5F002396E0238ACC2
:20396E007F011201CCE0A3F5F0E0C5F07F030201E67FFF7EFF1201E8743F75F059C0E0C0AB
:20398E00F0120CF91581158174C075F0A2C0E0C0F0745375F059C0E0C0F0E52B75F000C051
:2039AE00E0C0F0E52CC0E0C0F0E52D75F000C0E0C0F07405124A9C7FF612004F74C075F061
:2039CE00A2C0E0C0F0120CF91581158174C075F0A2C0E0C0F0747D75F059C0E0C0F0E52E07
:2039EE0075F000C0E0C0F0E5248525F0C0E0C0F0E50A75F000C0E0C0F07405124A9C7FF687
:203A0E0012004FE4F50A74C075F0A2C0E0C0F0120CF91581158174C075F0A2C0E0C0F07487
:203A2E00A375F059C0E0C0F0740275F000124A9C158115811581158174C075F0A2C0E0C001
:203A4E00F0120CF915811581E47F001201CCF07F001201CCE075F0007B067C0012017A7056
:203A6E0013023AE27F001201CCE0047F001201CCF01480DB74C075F0A2C0E0C0F074B475E0
:203A8E00F059C0E0C0F0E52B75F0007B067C001200B97F001201CC1200652BC5F03400C594
:203AAE00F0797F7AA412007789828A83E075F000C0E0C0F0740375F000124A9C7FFA12005D
:203ACE004F74C075F0A2C0E0C0F0120CF915811581023A7274C075F0A2C0E0C0F074BA75DF
:203AEE00F059C0E0C0F0740275F000124A9C158115811581158174C075F0A2C0E0C0F01257
:203B0E000CF915811581E47F001201CCF07F001201CCE075F0007B067C0012017A70130282
:203B2E003BA07F001201CCE0047F001201CCF01480DB74C075F0A2C0E0C0F074CC75F05914
:203B4E00C0E0C0F0E52C75F0007B067C001200B97F001201CC1200652BC5F03400C5F079B2
:203B6E007F7AA412007789828A83E075F000C0E0C0F0740375F000124A9C7FFA12004F7442
:203B8E00C075F0A2C0E0C0F0120CF915811581023B3074C075F0A2C0E0C0F074D275F059C1
:203BAE00C0E0C0F0740275F000124A9C158115811581158174C075F0A2C0E0C0F0120CF9DA
:203BCE0015811581E47F001201CCF07F001201CCE075F0007B067C0012017A7013023C5338
:203BEE007F001201CCE0047F001201CCF01480DB74C075F0A2C0E0C0F074E475F059C0E077
:203C0E00C0F0E5248525F07F001201CC1200652BC5F03400C5F0F9AAF089828A83E075F0B5
:203C2E0000C0E0C0F0740375F000124A9C7FFA12004F74C075F0A2C0E0C0F0120CF9158140
:203C4E001581023BEE74C075F0A2C0E0C0F074EA75F059C0E0C0F0740275F000124A9C15B6
:203C6E008115811581158174C075F0A2C0E0C0F0120CF915811581E47F001201CCF07F0074
:203C8E001201CCE075F0007B047C0012017A7013023CF87F001201CCE0047F001201CCF021
:203CAE001480DB74C075F0A2C0E0C0F074FC75F059C0E0C0F07F001201CCE079277A0075B1
:203CCE00F000120077E775F000C0E0C0F07403124A9C7FFA12004F74C075F0A2C0E0C0F0ED
:203CEE00120CF915811581023CA1740A75F000C0E0C0F0120B951581158174C075F0A2C088
:203D0E00E0C0F0740275F05AC0E0C0F0E53275F000C0E0C0F0E533C0E0C0F0E53475F000CE
:203D2E00C0E0C0F0E535C0E0C0F0740675F000124A9C7FF412004F74C075F0A2C0E0C0F085
:203D4E00120CF91581158174C075F0A2C0E0C0F0743575F05AC0E0C0F0E53275F000C3335D
:203D6E00C5F033C5F079737AAA12007789828A83E0A3F5F0E0C0F0C0E0740375F000124A17
:203D8E009C7FFA12004F74C075F0A2C0E0C0F0120CF91581158174C075F0A2C0E0C0F074D2
:203DAE004975F05AC0E0C0F0E53375F000C333C5F033C5F079737AAA12007789828A83E0FC
:203DCE00A3F5F0E0C0F0C0E0740375F000124A9C7FFA12004F74C075F0A2C0E0C0F0120CC6
:203DEE00F915811581740A75F000C0E0C0F0120B951581158174C075F0A2C0E0C0F0745D23
:203E0E0075F05AC0E0C0F0E52275F000C0E0C0F0E523C0E0C0F0E51575F000C0E0C0F0E5DD
:203E2E0014C0E0C0F0E51675F000C0E0C0F0E517C0E0C0F0740875F000124A9C7FF01200BA
:203E4E004F74C075F0A2C0E0C0F0120CF915811581E4F52EF5357F010201E6742C75F00197
:203E6E00C0E0C0F01246D415811581227FFC7EFF1201E8E4F5F07F001201CCF0A3C5F0F018
:203E8E00C5F0E47F021201CCF07F021201CCE075F0007B107C0012017A7012023F4E7F0260
:203EAE001201CCE0047F021201CCF080DCE47F031201CCF07F031201CCE075F0007B107CA3
:203ECE000012017A7012023F4B7F031201CCE0047F031201CCF080DC7F021201CCE075F0A2
:203EEE00007B207C001200B9C0E0C0F07F031201CCE075F000C333C5F033C5F0D004D003A2
:203F0E002BC5F03CC5F079BB7AAC12007789828A83E0A3F5F0E0C5F045F07003023F487F1A
:203F2E00001201CCE0A3F5F0E0C5F01201267F001201CCF0A3C5F0F0C5F0023ED7023EAC10
:203F4E007F001201CCE0A3F5F0E0C5F07F040201E67FFD7EFF1201E8E47F001201CCF07FE7
:203F6E00001201CCE075F0007B107C0012017A701202411C7F001201CCE0047F001201CCFA
:203F8E00F080DC74017F021201CCF0E47F011201CCF07F011201CCE075F0007B107C001212
:203FAE00017A70120240FE7F011201CCE0047F011201CCF080DC7F001201CCE075F0007BAA
:203FCE00207C001200B9C0E0C0F07F011201CCE075F000C333C5F033C5F0D004D0032BC54E
:203FEE00F03CC5F079BB7AAC12007789828A83E0A3F5F0E0C5F045F070030240FB7F021262
:20400E0001CCE0700302405B74C075F0A2C0E0C0F0749F75F05AC0E0C0F07F001201CCE0EA
:20402E00244175F000C0E0C0F0740375F000124A9C7FFA12004F74C075F0A2C0E0C0F0120D
:20404E000CF915811581E47F021201CCF074C075F0A2C0E0C0F074A475F05AC0E0C0F07FBC
:20406E00011201CCE0240175F000C0E0C0F0740375F000124A9C7FFA12004F74C075F0A2AF
:20408E00C0E0C0F0120CF9158115817F001201CCE075F0007B207C001200B9C0E0C0F07F2B
:2040AE00011201CCE075F000C333C5F033C5F0D004D0032BC5F03CC5F079BB7AAC120077DF
:2040CE0089828A83E0A3F5F0E0C5F07B087C00120114C0E0C0F01228831581158174207555
:2040EE00F000C0E0C0F0120B9515811581023FB57F021201CCE06003024119740A75F000BC
:20410E00C0E0C0F0120B9515811581023F827F030201E67FFB7EFF1201E890AEBBE0540412
:20412E0075F0007B007C001201717F021201CCF078F9120043E60886F090446B02009074D2
:20414E000175F000C0E0C0F078F9120043E60886F0C0E0C0F0124C8A1581158115811581E1
:20416E0078FB120043F608A6F0181818E60886F0541FC5F05400C5F07B087C0012010608D8
:20418E0046C5F00846C5F07F001201CCF0A3C5F0F0C5F078F5120043E60886F07B207C008B
:2041AE001200B9C0E0C0F008E60886F0C333C5F033C5F0D004D0032BC5F03CC5F079BB7AB1
:2041CE00AC12007789828A83E0A3F5F0E0C5F045F0700302424E78F5120043E60886F07BAC
:2041EE00207C001200B9C0E0C0F008E60886F0C333C5F033C5F0D004D0032BC5F03CC5F083
:20420E0079BB7AAC12007789828A83E0A3F5F0E0C5F07F001201CC120069120169700302CE
:20422E00423AE47F021201CCF002424B74A875F05A7F031201CCF0A3C5F0F0C5F002425F65
:20424E0074B075F05A7F031201CCF0A3C5F0F0C5F078F5120043E60886F07B207C001200D0
:20426E00B9C0E0C0F008E60886F0C333C5F033C5F0D004D0032BC5F03CC5F079BB7AAC1244
:20428E0000777F001201CCE0A3F5F0E0C5F089828A83F0A3C5F0F0C5F002448378F51200F1
:2042AE0043E60886F07B207C001200B9C0E0C0F008E60886F0C333C5F033C5F0D004D00371
:2042CE002BC5F03CC5F079BB7AAC12007789828A83E0A3F5F0E0C5F045F070030243407862
:2042EE00F5120043E60886F07B207C001200B9C0E0C0F008E60886F0C333C5F033C5F0D001
:20430E0004D0032BC5F03CC5F079BB7AAC120077E4F5F089828A83F0A3C5F0F0C5F074B40E
:20432E0075F05A7F031201CCF0A3C5F0F0C5F0024347E47F021201CCF0024483E4F5F07898
:20434E00F7120043F608A6F078F7120043E60886F07B107C0012017A701602445778F7120F
:20436E000043E60886F012012618F608A6F080D878F5120043E60886F07B207C001200B943
:20438E00C0E0C0F008E60886F0C333C5F033C5F0D004D0032BC5F03CC5F079BB7AAC1200DC
:2043AE007789828A83E0A3F5F0E0C5F045F0700302445478F5120043E60886F07B207C00E4
:2043CE001200B9C0E0C0F008E60886F0C333C5F033C5F0D004D0032BC5F03CC5F079BB7A8F
:2043EE00AC120077E4F5F089828A83F0A3C5F0F0C5F07F021201CCE0700302445474C075B6
:20440E00F0A2C0E0C0F074BC75F05AC0E0C0F078F1120043E60886F02441C5F03400C0F04D
:20442E00C0E0740375F000124A9C7FFA12004F74C075F0A2C0E0C0F0120CF915811581E46E
:20444E007F021201CCF002436BE47F021201CCF0024483E47F021201CCF00244834A4310B7
:20446E0000AA421500AA4214004D4113004D411200000061447F021201CCE07003024593BA
:20448E007F031201CCE0A3F5F0E0C0F0C0E0120CF91581158174D275F05AC0E0C0F0120C5F
:2044AE00F91581158178F5120043E60886F0C0E0C0F01227BE1581158174D875F05AC0E085
:2044CE00C0F0120CF91581158178F7120043E60886F0C0E0C0F01228281581158174DC7510
:2044EE00F05AC0E0C0F0120CF91581158178F9120043E60886F0C0E0C0F01228281581154A
:20450E008174C075F0A2C0E0C0F074E075F05AC0E0C0F078F7120043E60886F0C0E0C0F0A6
:20452E00740375F000124A9C7FFA12004F74C075F0A2C0E0C0F0120CF91581158178F71270
:20454E000043E60886F0C0E0C0F012288315811581742075F000C0E0C0F0120B95158115C7
:20456E008178F9120043E60886F0C0E0C0F01228831581158174EC75F05AC0E0C0F0120CBC
:20458E00F9158115817F050201E678F9120043E60886F07B207C001200B9C0E0C0F008E631
:2045AE000886F0C333C5F033C5F0D004D0032BC5F03CC5F079BB7AAC12007789828A83E089
:2045CE00A3F5F0E0C5F045F070030246A990AEBBE0540475F0007B007C0012017170030291
:2045EE00466A74C075F0A2C0E0C0F074EF75F05AC0E0C0F0740275F000124A9C1581158101
:20460E001581158174C075F0A2C0E0C0F0120CF91581158178F9120043E60886F0C0E0C008
:20462E00F01227BE1581158174FA75F05AC0E0C0F0120CF91581158178FB120043E608865D
:20464E00F0C0E0C0F012282815811581740A75F000C0E0C0F0120B951581158178F91200EA
:20466E0043E60886F07B207C001200B9C0E0C0F008E60886F0C333C5F033C5F0D004D003AD
:20468E002BC5F03CC5F079BB7AAC120077E4F5F089828A83F0A3C5F0F0C5F02278FB1200E3
:2046AE0043E60886F090ACB5F0A3C5F0F0C5F0E4F5F090ACB7F0A3C5F0F0C5F0E490ACBAE4
:2046CE00F090ACB9F02278FB120043E60886F0C0E0C0F01246AA1581158174BB75F0ACC02B
:2046EE00E0C0F0E4C0E0C0E0E475F002C0E0C0F0124BC57FFA02005E7FFA7EFF1201E8E48D
:20470E00F5F07F041201CCF0A3C5F0F0C5F090ACBAE00490ACBAF0540F90ACBAF0600302E9
:20472E00473F90ACB9E00490ACB9F0540F90ACB9F07F041201CCE0A3F5F0E0C5F012012647
:20474E007F041201CCF0A3C5F0F0C5F07B007C0112019060030247A990ACB9E075F0007B57
:20476E00207C001200B9C0E0C0F090ACBAE075F000C333C5F033C5F0D004D0032BC5F03CE3
:20478E00C5F079BB7AAC12007789828A83E0A3F5F0E0C5F045F0700302471C90ACB9E07507
:2047AE00F0007B207C001200B9C0E0C0F090ACBAE075F000C333C5F033C5F0D004D0032B29
:2047CE00C5F03CC5F079BB7AAC12007789828A83E0A3F5F0E0C5F045F0700302489390AC6C
:2047EE00B9E075F0007B207C001200B9C0E0C0F090ACBAE075F000C333C5F033C5F0D004D9
:20480E00D0032BC5F03CC5F079BB7AAC12007789828A83E0A3F5F0E0C5F05400C5F0541F72
:20482E00C5F07B087C001201147F001201CCF0A3C5F0F0C5F090ACB9E075F0007B207C00F3
:20484E001200B9C0E0C0F090ACBAE075F000C333C5F033C5F0D004D0032BC5F03CC5F07970
:20486E00BB7AAC12007789828A83E0A3F5F0E0C5F054FFC5F05400C5F07F021201CCF0A3A7
:20488E00C5F0F0C5F07F060201E67FFC7EFF1201E890ACB7E0A3F5F0E0C5F012012690ACEA
:2048AE00B7F0A3C5F0F0C5F090ACB5E0A3F5F0E0C5F045F0700302494F123E7A7F021201B8
:2048CE00CCF0A3C5F0F0C5F07F021201CCE0A3F5F0E0C5F045F0700302494C740175F0009B
:2048EE00C0E0C0F090ACB5E0A3F5F0E0C5F07F021201CC1200691200D3C0E0C0F0124C8A74
:20490E0015811581158115817F001201CCF0A3C5F0F0C5F090ACB7E0A3F5F0E0C5F07F0077
:20492E001201CC120069120190700302494C124706E4F5F090ACB7F0A3C5F0F0C5F002490F
:20494E005CE4F5F090ACB7F0A3C5F0F0C5F07F040201E67FFC7EFF1201E81201F31222FAB1
:20496E00120200D2AF12088E123E6990A38BE060030249D274FE75F05AC0E0C0F0120CF97D
:20498E0015811581742A75F05BC0E0C0F0120CF915811581743C75F05BC0E0C0F0120CF915
:2049AE0015811581744275F05BC0E0C0F0120CF915811581744875F05BC0E0C0F0120CF9D1
:2049CE00158115811212BA740175F00045F07003024A76E4A21792E0F51F70030249F8B2F0
:2049EE0097B297B297C21712489812290C7F021201CCF0A3C5F0F0C5F07BFF7CFF120171A8
:204A0E007003024A4090ACB4E0540175F0007B017C001201697003024A3D7F021201CCE04F
:204A2E00A3F5F0E0C0F0C0E0122ADC158115810249F8120FCC7F001201CCF0A3C5F0F0C5E1
:204A4E00F07B007C001201717003024A737F001201CCE0A3F5F0E0C0F0C0E012178B15816B
:204A6E0015811212BA0249D5747075F05BC0E0C0F0120CF9158115817F040201E623F425B5
:204A8E0081F81201B4124DC71201B402045923F42581F8868208868308024DC70000000090
:204AAE000000000000202020202000000000000000000000000000000000000060010101E5
:204ACE0001010101010101010101010118181818181818181818010101010101010A0A0AA7
:204AEE000A0A0A02020202020202020202020202020202020202020101010101010C0C0C38
:204B0E000C0C0C04040404040404040404040404040404040404040101010100C2D578FB05
:204B2E00120043E6904AAAC2E79355F060027401A2D575F00092F065F075F0002278FB1291
:204B4E000043E6A2E7B3E4F5F092E02275F00280CB75F00480C675F00680C175F01680BCC1
:204B6E0075F01780B775F05780B2D2D575F05780AD75F01080A675F00880A175F001809C4B
:204B8E0075F020809778FB120043E6C0E008E6C0E0124B5F13D0F0D0E0500224E02278FB65
:204BAE00120043E6C0E008E6C0E0124B5A13D0F0D0E050E924202278F7120043868208864B
:204BCE008308860708088603088604EB4C600AEFF0A31BBBFFF51C80F22278FB1200438699
:204BEE0082088683E4FBFCFFE0A3B42D030FE0A3C39430B40A005012FA740A75F0001200AB
:204C0E00B92AFBE5F03400FC80E4EB8CF0DF0302013E2278F91200438682088683E0600D67
:204C2E00A380FA78F91200438682088683088601088602C9C582C9CAC583CAE0A3C9C58203
:204C4E00C9CAC583CAF06003A380E8E5828583F02278FB1200438682088683E4F5F0FAE03E
:204C6E006009A30ABA00F805F080F4EA2278FB120043E60886F030F73A02013E78F9120098
:204C8E00438603088604088605088606ED8EF0120196401CED8EF02278F91200438603082D
:204CAE008604088605088606ED8EF012019640E4EB8CF02278FB120043860308860485FE0E
:204CCE00F0E5017F0012017A600575F001E422EF0FF5F0A412017A70F6EF1475F000227897
:204CEE00F91200438682088683088601088602C9C582C9CAC583CAE0F5F0A3C9C582C9CA60
:204D0E00C583CAE0B5F0056009A380E37401500274FF02008778F71200438601080886F0E6
:204D2E0008088603088604EB4C600AA7F0091BBBFFF51C80F222124D9E124DAA124DB11257
:204D4E004DB8E0F7A30980F7124D9E124DB1124DAA124DB8E7F009A380F7124D9E124DAA19
:204D6E00124DB1A882124DB8E6F7080980F7124D9E124DAA124DB1124DB8E0A3CAC583CAE3
:204D8E00C9C582C9F0A3CAC583CAC9C582C980E778FA1200438604188603182286831886AA
:204DAE0082182286021886011822EB4C60061BBBFF011C221581158122124F0E86820886C4
:204DCE008308E4FEFFE07006124F0EE4F022B42551A3E0B42D05430780A3E0B4300343078D
:204DEE004024D0B40A00500BCE75F00AA42EFEA3E080EEE0B46413E60886F030F708430772
:204E0E002012013EA6F018F68003B4750543070A8021B478054307108019B46F1043070820
:204E2E008011124F0EF0A3124F0EA38095B462624307027A00C004C005C006C007AB075351
:204E4E00031F7C00E60886F01200D3A6F018F6EDD007D006D005D0042430B43A00400224CE
:204E6E0007C0E00AE645F070CC124F0EA902EF30E505742DF0A30A124F17D0E0F0A3D9FA2D
:204E8E000808EF30E7A1EAC39E509C7420F0A30A80F4B4630DAA01124F0E124F17E6F0A342
:204EAE0080DEB47331C082C08386820886837A00E06004A30A80F98683188682124F0E1202
:204ECE004F17124F0EE0A3124F0E6004F0A380F2D005D00480AAB4691B86017A00E760043D
:204EEE00090A80F9124F0E124F178601E76091F009A380F8F97A01124F0E124F17E9809E5C
:204F0E00CDC583CDCCC582CC22EE601A8FF020F715C002EAC39E500C742030F6027430F0D4
:204F2E00A30A80EFD002224CFE4BFEB1F94CFE4BFEB1F94CFE4BFEA5FB24FE4CFE4BFEB140
:204F4E00F94CFE4BFEB1F94CFE4BFE99FDBCF630F818FCE000000006900000060A900000E0
:204F6E000E0590000002099000000A0560000001096000000906600000050A6000000D061B
:204F8E00A00000070AA000000F05A000000309A000000B055000000009500000080650003B
:204FAE0000040A5000000C4D45434B4F4741494E46444C5048424A00000694000C000A94AD
:204FCE00001C0005940004000994001400056400020009640012000664000A000A64001A73
:204FEE000006A4000E000AA4001E0005A400060009A40016000554000000095400100006E1
:20500E00540008000A5400180005580001000568000300059800050005A80007000658002E
:20502E0009000668000B000698000D0006A8000F00095800110009680013000998001500CC
:20504E0009A80017000A580019000A68001B000A98001D000AA8001F0C10041102120A1380
:20506E000E140615001608170D180519031A0B1B0F1C071D011E091F5751605169517251BE
:20508E007B5184518D5196519F51A851B251BC51C651D051DA51E451EE51FC510A520D52C4
:2050AE00115215521C522B52395246525752645271527F528C529A52303100303200303327
:2050CE000030340030350030360030370030380030390031300031310031320031330031A0
:2050EE003400313500313600414600414E004F4E004F4600444D004252004C460058430007
:20510E00485200484100504400504400584400534E0053460053520000010203040506079F
:20512E0008090A0B0C0D0E0F101112131415161718191A1B1C1D1E1FA952AC52AF5258300B
:20514E00310058313020003353446576696365203100446576696365203200446576696383
:20516E00652033004465766963652034004465766963652035004465766963652036004436
:20518E006576696365203700446576696365203800446576696365203900446576696365FD
:2051AE0020313000446576696365203131004465766963652031320044657669636520311A
:2051CE0033004465766963652031340044657669636520313500446576696365203136000C
:2051EE00416C6C20556E697473204F666600416C6C204C6967687473204F6E004F6E004F8D
:20520E0066660044696D0042726967687400416C6C204C6967687473204F6666004578742A
:20522E00656E64656420436F6465004861696C2052657175657374004861696C2041636B91
:20524E006E6F776C65646765005072657365742044696D2030005072657365742044696D41
:20526E00203100457874656E646564204461746100537461747573206973204F6E005374E0
:20528E0061747573206973204F6666005374617475732052657175657374005858004F463A
:2052AE00004F4E00436F6E736F6C652073746174757320666C61677320253032780A002036
:2052CE005472616E733A20204865616420253032782C205461696C20253032782C204374B5
:2052EE007220253032782C204D617820253032780A00205265633A202020204865616420EE
:20530E00253032782C205461696C20253032782C2043747220253032782C204D6178202540
:20532E003032780A0030313233343536373839414243444546003030200020002A2A2A209B
:20534E0042616420636865636B73756D3A202532780A002A000A002A2120004F4B0A003E11
:20536E00002A2A2A204E6F206164647265737320737472696E672E2E2E0A004E65742061CB
:20538E006464726573732069732025730A004E65742061646472657373205B25735D002EF1
:2053AE002020537461636B207573656420253032782F253032782E0A004572726F722066C3
:2053CE006C61677320253032782E20204E6574776F726B20636865636B73756D20657272C5
:2053EE006F72732025750A004C6F6767696E67206D6F64652069732025750A004E657420F4
:20540E006D6F64652069732025750A002A2A2A204E20636D642073796E74617820657272A9
:20542E006F720A002A2A2A20556E6B6E6F776E20636F6D6D616E643A205B25735D0A004DE5
:20544E00616E75616C2072656D6F746520696E707574206D6F64652069732025750A004666
:20546E0061696C3D25752C0025750A002A2A2A205120636D642073796E74617820657272CE
:20548E006F720A0052656672657368206379636C6520257520736563207769746820257569
:2054AE00206D6F64756C65730A0045534554002A2A2A20556E6B6E6F776E20636F6D6D61CF
:2054CE006E640A002A2A2A205220636D642073796E746178206572726F720A002A2A2A20E5
:2054EE005320636D642073796E746178206572726F720A00417661696C61626C6520636F69
:20550E006D6D616E6473202876616C7565732061726520646563696D616C20756E6C657397
:20552E0073206E6F746564290A0020413D737472696E6720202B2020736574206E65747773
:20554E006F726B20616464726573730A0020442020202020202020202A202064756D70201D
:20556E00696E7465726E616C20737461747573207661726961626C657320286D6F737420F8
:20558E00696E20686578290A0020452020202020202020202A202064756D7020616E642076
:2055AE00636C656172206572726F7220666C6167730A00204620202020202020202020208F
:2055CE0020666C757368207472616E732F72656320627566666572730A00204C206E202079
:2055EE002020202020202020736574207265706F7274696E67206D6F646573202862697498
:20560E006D6170706564290A00204D206E20202020202020202020736574206D616E756119
:20562E006C2072656D6F746520636F6E74726F6C206D6F64650A00204E206E2020202020B8
:20564E0020202B2A20736574206E6574776F726B206D6F64650A00205020202020202020F2
:20566E002020202020646973706C617920616E6420636C65617220706F776572206661696F
:20568E006C207374617475730A00205120202020202020202020202064756D7020616C6CC2
:2056AE00206D6F64756C65730A00205120682020202020202020202064756D7020616C6C71
:2056CE00206D6F64756C657320666F7220686F757365636F64650A0020512068206D6D2040
:2056EE0020202020202064756D702073696E676C65206D6F64756C6520666F7220686F750B
:20570E007365636F64650A00205120532020202020202020202064756D7020616C6C206D3E
:20572E006F64756C657320696E206865780A00205220202020202020202020202064756D31
:20574E0070207265667265736820696E74657276616C0A002052206E20202020202020202D
:20576E002020736574207265667265736820696E206D696E757465730A0020522043206EF7
:20578E002020202020202020636C6561722072656672657368206275666665722C20736527
:2057AE007420696E206D696E757465730A0020522053206E20202020202020207365742062
:2057CE007265667265736820696E207365636F6E64730A00205220512020202020202020D9
:2057EE00202064756D702072656672657368207461626C6520656E74726965730A002052D8
:20580E00455345542020202020202020706572666F726D20706F7765722D6F6E207265738D
:20582E00657420696E697469616C697A6174696F6E0A0020532068206D6D20636320727290
:20584E002073656E6420636F6D6D616E6420746F206D6F64756C6520617420686F7573658F
:20586E00636F64650A004D6F64756C6573206D7573742062652073706563696669656420E0
:20588E00776974682074776F206469676974733A202053204E203037204F4E0A002B206DDF
:2058AE0061726B73206E6574776F726B2D6F6E6C7920636F6D6D616E64730A002A206D617C
:2058CE00726B7320646562756767696E6720636F6D6D616E64730A0025633D25303278005E
:2058EE0025303278002573005263763A2020483D0020442F463D00202800290A00253034BF
:20590E00780025633D002563253032753D25730A00456E513A2020483D0020443D002046CF
:20592E003D00205265703D252D3275202800290A00506F776572206C696E65207374617473
:20594E0075733A0A00205472616E733A20204865616420253032782C205461696C2025308F
:20596E0032782C2043747220253032782C20004D617820253032782C204F75745074722070
:20598E00253034782C20457272466C61677320253032780A0020205B584F757448656164D0
:2059AE005D202D3E20002025303278000A20205B584F75745461696C5D202D3E20002025A6
:2059CE00303278000A20205B584F75745074725D20202D3E20002025303278000A2020588B
:2059EE004F7574426974735B5D202D3E2000202530327800205265633A202020204865614B
:205A0E006420253032782C205461696C20253032782C2043747220253032782C204D6178FA
:205A2E0020253032780A0020205B58496E486561645D202D3E20253034780020205B5849CE
:205A4E006E5461696C5D202D3E20253034780020506F7765726661696C3A202041434269C5
:205A6E007473202530327820253032782C2073746174652025752C206379632025752C203B
:205A8E00676F6F642025752C206261642025750A0025633A200025753D00436867205265BC
:205AAE00660052656600436C722052656600436C7220416C6C2072656620666F7220483D34
:205ACE0025630A003A2020483D0020443D0020463D00205265703D252D3275202800290AEB
:205AEE000044656C2072656620483D0020443D000A504C2D4C696E6B204E6574776F726B75
:205B0E0065642058313020436F6E74726F6C6C65722C2056657273696F6E2000312E32644A
:205B2E0020286E6F2072656672657368290020666F722000363020487A000A2020436F70BF
:205B4E00797269676874203139393220436972637569742043656C6C61722C20496E632EB1
:1C5B6E000A002D2D2D2046656C6C206F75742074686520626F74746F6D210A002E
:00000001FF
